S021000064656D6F70726F675F6F6C696D65785F73746D3332703130332E737265639D
S3150800600008090020517B0008A97B0008AD7B000821
S31508006010B17B0008B57B0008B97B000800000000CA
S31508006020000000000000000000000000BD7B000822
S31508006030C17B000800000000C57B00086F750008DA
S31508006040C97B0008CD7B0008D17B0008D57B0008FA
S31508006050D97B0008DD7B0008E17B0008E57B0008AA
S31508006060E97B0008ED7B0008F17B0008F57B00085A
S31508006070F97B0008FD7B0008017C0008057C000808
S31508006080097C00080D7C0008117C0008157C0008B6
S31508006090197C00081D7C0008217C0008257C000866
S315080060A0297C00082D7C0008317C0008357C000816
S315080060B0397C00083D7C0008417C0008457C0008C6
S315080060C0497C00084D7C0008517C0008557C000876
S315080060D0597C00085D7C0008617C0008657C000826
S315080060E0697C00086D7C0008717C0008EE11AA55D1
S315080060F02DE9FC41040000202078C0076BD5DFF8A5
S31508006100C005016811F00C01042907D0016811F0D7
S315080061100C0108290CD10068C00309D5DFF89C05D5
S315080061200068800357D56068002854D10120B3E180
S315080061306068B0F5803F06D1DFF88005016851F444
S315080061408031016026E0606800280AD1DFF86C0516
S31508006150016831F480310160016831F48021016001
S3150800616018E06068B0F5A02F0AD1DFF8500501687D
S3150800617051F480210160016851F48031016009E021
S31508006180DFF83805016831F480310160016831F4BF
S3150800619080210160606800280ED000F0B1FA050081
S315080061A0DFF818050068800315D400F0A9FA401B2B
S315080061B06528F5D303206FE100F0A2FA0500DFF8A1
S315080061C0FC040068800306D500F09AFA401B65288F
S315080061D0F5D3032060E1207880071ED5DFF8E004B8
S315080061E0016811F00C0F07D0016811F00C0108299D
S315080061F02CD10068C00329D4DFF8C00401688907D8
S3150800620004D52169012901D0012045E1016831F051
S31508006210F801626951EAC20101602078000749D590
S31508006220A069002871D00120DFF8A414086000F0E6
S3150800623067FA0500DFF894040068800737D400F091
S315080062405FFA401B0328F5D3032025E120690028BF
S315080062501AD00120DFF87C14086000F051FA050016
S31508006260DFF858040168890706D400F049FA401B8C
S315080062700328F5D303200FE1016831F0F8016269BC
S3150800628051EAC2010160C8E70020DFF84814086037
S3150800629000F036FA0500DFF8240400688007BCD54C
S315080062A000F02EFA401B0328F5D30320F4E0012062
S315080062B000F0F0F92078400740F196800026DFF8D4
S315080062C018542868C00009D4286850F080502860FF
S315080062D0286810F08050009000980126DFF8FC73BB
S315080062E03868C00524D4386850F48070386000F0E7
S315080062F007FA80463868C0051AD400F001FAB0EBF0
S3150800630008006528F6D30320C6E00020DFF8C0138E
S31508006310086000F0F5F90500DFF8B00300688007AB
S31508006320C8D500F0EDF9401B0328F5D30320B3E0E8
S31508006330E068012806D1DFF8A803016851F00101D9
S31508006340016025E0E06800280AD1DFF894030168B7
S31508006350490849000160016831F00401016017E04D
S31508006360E06805280AD1DFF87803016851F00401CE
S315080063700160016851F00101016009E0DFF860037E
S315080063800168490849000160016831F004010160AB
S31508006390E068002810D000F0B3F90700DFF84003E2
S315080063A00068800719D400F0ABF9C01B41F28931A7
S315080063B08842F3D303206FE000F0A2F90700DFF864
S315080063C020030068800708D500F09AF9C01B41F23F
S315080063D089318842F3D303205EE0F6B2012E03D159
S315080063E0286830F080502860E069002853D0DFF82C
S315080063F0D062306810F00C0008284AD0E0690228FC
S3150800640034D1DFF8E0720020386000F079F9804670
S31508006410DFF8A8522868800107D500F071F9B0EBBB
S3150800642008000328F4D3032036E0206AB0F5803F3D
S3150800643005D1316831F40031A06801433160316813
S3150800644031F47411206A0143606A01433160012006
S31508006450386000F055F90400286880011BD400F064
S315080064604FF9001B0328F7D3032015E00020DFF8B7
S315080064707412086000F044F90400DFF8400200686E
S31508006480800108D500F03CF9001B0328F5D303204A
S3150800649002E0012000E00020BDE8F6812DE9F04188
S315080064A004000D000020DFF84062306810F0070095
S315080064B0A8420BD23068C008C00028433060306854
S315080064C010F00700A84201D0012097E02078800745
S315080064D007D5DFF8EC110A6832F0F002A06802432B
S315080064E00A602078C00754D56068012806D1DFF80D
S315080064F0CC010068800310D401207FE06068022880
S3150800650005D16E480068800107D4012076E06B4803
S315080065100068800701D4012070E0694F396889084E
S31508006520890060680143396000F0EAF880466068CF
S3150800653001280ED1386810F00C00042829D000F084
S31508006540DFF8B0EB080041F289318842F2D3032024
S3150800655054E0606802280ED1386810F00C0008284C
S3150800656017D000F0CDF8B0EB080041F28931884227
S31508006570F2D3032042E0386810F00C0F09D000F07F
S31508006580BFF8B0EB080041F289318842F3D3032003
S3150800659034E0306810F0070085420BD23068C00836
S315080065A0C00028433060306810F00700A84201D0C8
S315080065B0012023E02078400706D541490A6832F4CD
S315080065C0E062E06802430A602078000707D53C4885
S315080065D0016831F46051226951EAC201016000F094
S315080065E00FF84249364A1268C2F30312895CC8405A
S315080065F035490860002000F089F80020BDE8F081E0
S3150800660000B585B001A83A49102200F0A5F8394826
S315080066100088ADF80000002000200020002000209F
S31508006620274A116811F00C00042802D0082802D065
S3150800663014E0244813E001A8C1F38343C05CC903EE
S3150800664009D569461268C2F340428A5C1D49484327
S31508006650B0FBF2F001E02849484300E0194805B0CC
S3150800666000BD19480068704780B5FFF7FAFF23494F
S31508006670134A1268C2F30222895CC84002BD80B57B
S31508006680FFF7EFFF1D490E4A1268C2F3C222895C62
S31508006690C84002BD81B00C490968C9084FF47A722E
S315080066A0B1FBF2F14843009000BF0098411E0091EB
S315080066B00028F9D101B07047000000000010024020
S315080066C00410024000127A00040000202410024040
S315080066D080044242000042421C1002400070004002
S315080066E0201002406000424200200240787B0008E9
S315080066F0687B00082272000800093D00A07B00089C
S3150800670001480068704700BF0001002010B504006A
S315080067104FF47A700D490978B0FBF1F00C49096815
S31508006720B1FBF0F000F0E6F8002801D001200CE0FB
S31508006730102C09D2002221005FF0FF3000F0C9F8C2
S3150800674004480460002000E0012010BD0800002075
S315080067500400002000000020103A07D330B4B1E846
S315080067603810103AA0E83810F9D230BC530724BFC5
S31508006770B1E80810A0E8081044BF51F8043B40F8F7
S31508006780043BD20724BF31F8022B20F8022B44BF62
S315080067900B7803707047121F17D35B0009D151F8A5
S315080067A0043B20F8023B1B0C121F20F8023BF6D2D2
S315080067B00BE051F8043B00F8013B1B0A20F8023BAA
S315080067C01B0C121F00F8013BF3D238BF121D521ED4
S315080067D024BF11F8013B00F8013BF8D8704730B4E4
S315080067E0002513E050F8042BD30744BFA9F1010391
S315080067F09A18091F042942F8045BFAD213468C0733
S3150800680044BF15809B1CC90748BF1D7050F8041B60
S315080068100029E7D130BC704710F007003E4B1A68D4
S315080068204FF6FF010A403D4951EA00210A431A6022
S31508006830704739480068C0F302207047020052B218
S31508006840002A08D50901364A40B210F00F00104454
S3150800685000F8041C03E00901324A40B2115470479B
S3150800686010B410F00700D0F10703052B01D3042359
S3150800687001E0D0F10703041D072C01D2002000E037
S31508006880C01E012414FA03F35B1E1940814014FA52
S3150800689000F0401E1040084310BC704780B5411EEA
S315080068A0B1F1807F01D301200EE0401E1E49086029
S315080068B00F215FF0FF30FFF7C1FF00201B4908607A
S315080068C007201B490860002002BD80B5FFF7A4FF1A
S315080068D001BD70B504000D0016000020FFF7A9FFE2
S315080068E032002900FFF7BCFF0100200040B2FFF785
S315080068F0A5FF70BD80B5FFF7D1FF02BD042805D1FD
S315080069000B48016851F00401016004E00848016879
S3150800691031F00401016070470CED00E00000FA0553
S3150800692018ED00E000E400E014E000E018E000E004
S3150800693010E000E080B500F001F801BD704730B402
S315080069400EE00268436802440830DC0744BFA9F138
S315080069500104E31852F8045B43F8045B091FF9D1F4
S3150800696050F8041B0029ECD130BC7047F8B5040078
S31508006970002500200026002C01D101209FE094F874
S315080069803C00002805D1002084F83D00200000F0D6
S3150800699090FA022084F83C002068006830F0020073
S315080069A0216808602068006850F0010021680860C6
S315080069B0FFF7A6FE070020684068C0070CD4FFF75B
S315080069C09FFEC01B0B28F6D3032084F83C0000204A
S315080069D084F83D00032072E020684068C00761D54E
S315080069E0A069012802D156F0800601E036F080063B
S315080069F0E069012802D156F0400601E036F040066B
S31508006A00206A012802D156F0200601E036F0200659
S31508006A10606A012802D156F0100601E036F0100629
S31508006A20A06A012802D156F0080601E036F00806E9
S31508006A30E06A012802D156F0040601E036F00406A1
S31508006A402068006830F0FC00064320680660A168EC
S31508006A50E068014320690143606901436068401E9C
S31508006A6001432068C1612068006840084000216829
S31508006A700860FFF745FE060020684068C0070CD589
S31508006A80FFF73EFE801B0B28F6D3032084F83C0054
S31508006A90002084F83D00032011E020684068C00704
S31508006AA000D40125012D06D100202064012084F898
S31508006AB03C00002003E0042084F83C000120F2BDDD
S31508006AC030B4002201224B6912FA03F30268D2F8A5
S31508006AD0002232F47C524C6A52EA042252F0010235
S31508006AE00468C4F800220268D2F81C229A43046893
S31508006AF0C4F81C22CA69002A1CD10268D2F80C22E2
S31508006B009A430468C4F80C2202684C6902EBC40272
S31508006B10CC684D68ADB255EA0445C2F840520268E1
S31508006B204C6902EBC4028C680D68ADB255EA04459F
S31508006B30C2F84452CA69012A1CD10268D2F80C224A
S31508006B401A430468C4F80C2202684C6902EBC402B2
S31508006B500C684D68ADB255EA0445C2F84052026861
S31508006B604C6902EBC4028C68CD68ADB255EA04459F
S31508006B70C2F844528A69002A07D10268D2F8042268
S31508006B809A430468C4F8042206E00268D2F804228C
S31508006B901A430468C4F804220A69002A07D102685D
S31508006BA0D2F814229A430468C4F8142206E002684C
S31508006BB0D2F814221A430468C4F81422096A01296F
S31508006BC006D10168D1F81C120B430168C1F81C32C2
S31508006BD00168D1F80012490849000068C0F8001297
S31508006BE0002030BC7047F8B505000E0014000020E0
S31508006BF000203000C0B2002811D195F83C002228A8
S31508006C000BD095F83C00422807D095F83C0062283E
S31508006C1003D095F83C00722801D1022048E13000E3
S31508006C20C0B2012811D195F83C0032280BD095F84E
S31508006C303C00522807D095F83C00622803D095F806
S31508006C403C00722801D1022032E195F83D00012866
S31508006C5001D102202CE1012085F83D003000C0B2A8
S31508006C60002818D195F83C00122804D0322806D0FE
S31508006C70522808D00BE0422085F83C0023E0622029
S31508006C8085F83C001FE0722085F83C001BE02220B6
S31508006C9085F83C0017E095F83C00122804D0222815
S31508006CA006D0422808D00BE0522085F83C000AE0BE
S31508006CB0622085F83C0006E0722085F83C0002E078
S31508006CC0322085F83C00FFF71BFD07003000C0B2F4
S31508006CD0002804D12868C06810F0030003E028687B
S31508006CE0006910F00300002811D114F1010FEDD04E
S31508006CF0002C04D0FFF704FDC01B8442E6D2032013
S31508006D0085F83C00002085F83D000320D0E03000DF
S31508006D10C0B2002801D1696B00E0A96B286832006F
S31508006D20D2B212011044D0F8B00110F00400886005
S31508006D308868002809D128683200D2B212011044A6
S31508006D40D0F8B001400D086008E028683200D2B2D9
S31508006D5012011044D0F8B001C00848602868320013
S31508006D60D2B212011044D0F8B00110F00200C86087
S31508006D7028683200D2B212011044D0F8B40110F0DB
S31508006D800F00086128683200D2B212011044D0F808
S31508006D90B401C0F30720C8613000C0B20862286891
S31508006DA03200D2B212011044D0F8B801087528682A
S31508006DB03200D2B212011044D0F8B801000A487560
S31508006DC028683200D2B212011044D0F8B801000C7B
S31508006DD0887528683200D2B212011044D0F8B8017A
S31508006DE0000EC87528683200D2B212011044D0F8D5
S31508006DF0BC01087628683200D2B212011044D0F8D5
S31508006E00BC01000A487628683200D2B21201104442
S31508006E10D0F8BC01000C887628683200D2B212017C
S31508006E201044D0F8BC01000EC8763000C0B2002865
S31508006E3003D120202968C86002E02020296808615B
S31508006E40F6B2002E18D195F83C00422804D06228E4
S31508006E5006D0722808D00BE0122085F83C0023E003
S31508006E60322085F83C001FE0522085F83C001BE0E4
S31508006E70012085F83C0017E095F83C00522804D01C
S31508006E80622806D0722808D00BE0122085F83C004C
S31508006E900AE0222085F83C0006E0422085F83C00FE
S31508006EA002E0012085F83C00002085F83D0000201E
S31508006EB0F2BD704710B50400002C01D1012033E063
S31508006EC0A0690028FFD194F83900002805D10020D0
S31508006ED084F83800200000F0A3F9242084F839004B
S31508006EE02068C06830F400502168C860200000F0AF
S31508006EF0C7F82068006930F4904021680861206866
S31508006F00406930F02A00216848612068C06850F45A
S31508006F1000502168C8600020E063202084F839000A
S31508006F20202084F83A00002010BD2DE9FC41050018
S31508006F300C0090461F00002095F83A00202865D1DD
S31508006F40002C03D0404680B2002801D101205EE023
S31508006F5095F83800012801D1022058E0012085F86B
S31508006F6038000020E863222085F83A00FFF7C8FBBE
S31508006F700600A5F82C80A5F82E8005E0286840684C
S31508006F80C005C00D0880A41CE88D002836D0E88D01
S31508006F90401EE885A868B0F5805F15D100973300D4
S31508006FA000222021280000F034F8002801D0032010
S31508006FB02DE0210028690028E0D02868406800F004
S31508006FC0FF000880641CDFE70097330000222021B9
S31508006FD0280000F01EF8002801D0032017E02869D1
S31508006FE0002804D1286840682070641CCCE728680B
S31508006FF0406810F07F002070641CC5E7202085F8E3
S315080070003A00002085F83800002000E00220BDE89C
S31508007010F6812DE9F04105000E0090461F00069CFA
S31508007020286800683040B04201D1012000E0002005
S315080070304146C9B2884220D114F1010FF0D0002C84
S3150800704004D0FFF75DFBC01B8442E9D22868C068FC
S3150800705030F4D0702968C860286840694008400044
S3150800706029684861202085F83900202085F83A00EB
S31508007070002085F83800032000E00020BDE8F081F4
S315080070802DE9F041040000212068026932F44052DB
S31508007090E068024320680261A268206902436069C9
S315080070A0024311432068C2685B48024011432068C6
S315080070B0C1602068416931F44071A06901432068C4
S315080070C0416120685549884251D1FFF7D8FA804670
S315080070D0FFF7D5FA0500FFF7D2FA0600FFF7CFFA51
S315080070E00700FFF7CCFA6421192202FB08F8636847
S315080070F09B00B8FBF3F35FF0640CB3FBFCF355435A
S31508007100D4F804C05FEA8C0CB5FBFCF55643D4F8FA
S3150800711004C05FEA8C0CB6FBFCF65FF0640CB6FBA9
S31508007120FCF601FB16552D0132356426B5FBF6F53E
S3150800713015F0F00515EB0315574363689B00B7FB7D
S31508007140F3F302FB00F260688000B2FBF0F0642201
S31508007150B0FBF2F001FB1031080132306421B0FBBC
S31508007160F1F010F00F0045192068856050E0FFF730
S315080071707BFA8046FFF778FA0500FFF775FA0600EE
S31508007180FFF772FA0700FFF76FFA6421192202FB6C
S3150800719008F863689B00B8FBF3F35FF0640CB3FB75
S315080071A0FCF35543D4F804C05FEA8C0CB5FBFCF538
S315080071B05643D4F804C05FEA8C0CB6FBFCF65FF0C5
S315080071C0640CB6FBFCF601FB16552D013235642618
S315080071D0B5FBF6F515F0F00515EB0315574363688F
S315080071E09B00B7FBF3F302FB00F260688000B2FB7A
S315080071F0F0F06422B0FBF2F001FB103108013230E6
S315080072006421B0FBF1F010F00F0045192068856085
S31508007210BDE8F08100000000F3E9FFFF00380140F7
S3150800722070470102BFF34F8FB7490A6812F4E0624C
S31508007230B64802430A60BFF34F8F00BFFDE780B52B
S3150800724000F00DF800F0C4F801BD80B500F01DF897
S3150800725000F028F901BD80B5FFF7E4FF01BD80B550
S31508007260AB48AC4901604FF461414160002181603F
S315080072700021C16000210161002181610C21416169
S315080072800021C161FFF716FE01BD70B5A24C20783A
S31508007290002815D1A14D280000F037F8012833D170
S315080072A02878002830D0287841282DDA00F05BF9B4
S315080072B09B4908600120207000209A49087023E045
S315080072C0984D964E28783044401C00F01EF8012848
S315080072D011D12878401C287028783178884213D133
S315080072E0002020707078FF280ED1287802280BD14C
S315080072F0FFF7B1FF08E000F036F9894909686431FB
S31508007300814201D20020207070BD80B501000023A3
S3150800731001227F48FFF709FEC0B2002801D10120EB
S3150800732000E0002002BDF8B504000D0016001F009D
S31508007330FFF79AF94FF47A71B0FBF1F2002300E0F7
S315080073405B1C1800C0B2122840D2DFF8DCC120004E
S3150800735080B21900C9B21CF811E01900C9B20CEBC9
S315080073604101497811EB0E0E1EF1010E0EFB00F0DD
S31508007370B2FBF0F100FB11200028E1D1210089B20F
S315080073801800C0B21CF810E01800C0B20CEB4000A0
S31508007390407810EB0E0E1EF1010E0EFB01F1B2FB4A
S315080073A0F1F0288028880028CAD0288840F20141B0
S315080073B08842C5DA1800C0B21CF810003070DBB27B
S315080073C00CEB430040783870012000E00020F2BD45
S315080073D078B58BB00020ADF8020000208DF80100CA
S315080073E000208DF8000040F267656B460DF101023A
S315080073F00DF102014FF4FA70FFF795FF4B4C4C4E16
S315080074002660002020634B4860630020A0610020AE
S31508007410E06100202062002060620020A062002057
S31508007420E0620020A0600020E0609DF80100401E98
S31508007430000420619DF80000401E00056061BDF84B
S31508007440020060602000FFF791FA002D02D46D0556
S31508007450394805E025F00045ED0055F004053748A4
S315080074602168B14202D10021069101E00E21069160
S3150800747000210791012108912900090C0191ADB25B
S3150800748002950100090C039180B204900020059032
S31508007490012009900E200A9001A92000FFF710FB91
S315080074A00CB070BD70B540F2676600251F4C00220F
S315080074B000212000FFF797FB002823D1002E09D4CE
S315080074C0606B0068B04210D1606B806800280CD1F0
S315080074D001250AE026F00046606B4068B04204D1F8
S315080074E0606B8068042800D10125EDB2012D09D111
S315080074F0606B007DFF2805D1606B0069022801D109
S31508007500FFF7A9FE70BD00000CED00E00400FA05C7
S315080075109400002000440040050100200C000020D3
S31508007520F800002004010020C07A0008500000205E
S3150800753000640040D40000200400E0FFFCFF1F00A8
S3150800754080B5FFF78EF84FF47A71B0FBF1F0FFF7CC
S31508007550D1F90420FFF7D2F9002200215FF0FF30AD
S31508007560FFF7B7F901BD80B5FFF7CAF802BD80B5C8
S3150800757000F004F8FFF7DEF901BD000003490A68C8
S315080075800348007882180A60704700BF000100208F
S315080075900800002080B500F007F8FFF750FE00F05D
S315080075A011F9FFF752FEFAE780B500F009F800F086
S315080075B031F900F009F8FFF7C3FF00F0FBF801BD49
S315080075C0744875490860704700B58FB0012005906A
S315080075D05FF480300690002107910121099102216C
S315080075E00C910D905FF4E0100E9005A8FEF780FD53
S315080075F0002800D0FEE70F2000900220019000200E
S3150800760002904FF48060039000200490022168469F
S31508007610FEF744FF002800D0FEE70FB000BD18B5FE
S3150800762085B05E48016851F001010160016811F0FA
S315080076300101049104995A490A6852F080520A6075
S315080076400A6812F080520492049A026852F0040200
S315080076500260026812F004020492049A026852F068
S3150800766008020260026812F008020492049A02688C
S3150800767052F010020260006810F01000049004989E
S31508007680086850F400300860086810F40030049068
S315080076900498086850F000700860086810F00070D8
S315080076A0049004980320FFF710F9002200217FF0C8
S315080076B00B00FFF70EF9002200217FF00A00FFF702
S315080076C008F9002200217FF00900FFF702F90022DD
S315080076D000217FF00400FFF7FCF8002200217FF06C
S315080076E00300FFF7F6F8002200217FF00100FFF7FC
S315080076F0F0F8002200215FF0FF30FFF7EAF84FF4B8
S3150800770080500090012001900020029002200390F2
S31508007710244C6946200000F08FF801224FF480516E
S31508007720200000F063F90420009002200190032055
S3150800773003901D4C6946200000F07EF80820009052
S3150800774000200190002002906946200000F074F89D
S315080077504FF4807000900020019000200290134C96
S315080077606946200000F068F84FF400700090022087
S315080077700190032003906946200000F05DF80C494B
S31508007780086830F4C04050F0E06050F4804008606B
S3150800779006B010BD0060000808ED00E018100240B1
S315080077A01C1002400010014000080140000C014076
S315080077B00400014080B501224FF48051124800F0C0
S315080077C015F901BD38B5FFF7CEFE04000F4D286840
S315080077D0201AB0F5FA7F15D30D490878002808D184
S315080077E00120087000224FF48051074800F0FEF887
S315080077F007E00020087001224FF48051024800F08B
S31508007800F5F82C6031BD000000100140FC00002096
S315080078100601002080B50748016851F01001016093
S315080078200320FFF752F80020FEF770FFFFF7F7FE78
S31508007830002002BD00200240F8B50200002000200A
S31508007840002000250020002314E0DFF8B4010668B4
S3150800785036EA040404600CE0DFF8A8010668A643CB
S31508007860066048688002F0D5DFF89401066834435C
S3150800787004605B1C102B80F0B88001269E400C68C3
S315080078803440B442F5D14868002827D001281AD0D8
S3150800789002281DD003282FD0112816D012281AD056
S315080078A0594FB8421AD0594FB84217D0584FB84214
S315080078B014D0584FB84211D0574FB8420ED0574F30
S315080078C0B8420BD01AE0CD6818E0CD682D1D15E03A
S315080078D0CD68083512E0CD680C350FE088680028B9
S315080078E001D1042507E08868012802D10825166118
S315080078F001E00825566101E00025FFE7B4F5807F21
S3150800790001D2170000E0171DB4F5807F02D25FEAA6
S31508007910830C03E0B3F1080C5FEA8C0C0F26D7F84A
S3150800792000E016FA0CF03EEA000E15FA0CFC5CEACA
S315080079300E0CC7F800C04868C0009AD538480768D2
S3150800794057F001070760006810F0010000900098E2
S31508007950344F1800800857F820C013F00300C0B24F
S31508007960800086403CEA060C2F48824201D1002658
S315080079700FE02E48824201D101260AE02C488242B5
S3150800798001D1022605E02B48824201D1032600E0F8
S31508007990042613F00300C0B28000864056EA0C0C99
S315080079A01800800847F820C04868C00304D5224854
S315080079B006682643066003E01F480668A643066075
S315080079C04868800304D51D4806682643066003E018
S315080079D01A480668A64306604868C0027FF53CAFA9
S315080079E008480668264306603BE7F1BDD2B2002A7E
S315080079F002D089B2016102E089B2090401617047C7
S31508007A000C04014008040140000011100000121087
S31508007A100000211000002210000031100000321072
S31508007A20181002400800014000080140000C0140FF
S31508007A300010014000140140000401400404014004
S31508007A400F49086850F0010008600E4A13680E488E
S31508007A50034013600B680D4803400B60086830F458
S31508007A6080200860106830F4FE0010605FF41F0084
S31508007A70074908605FF00060064908607047000023
S31508007A8000100240041002400000FFF8FFFFF6FE57
S31508007A900810024008ED00E010B50749794418318E
S31508007AA0064C7C44163404E00A68081D11448847CD
S31508007AB00146A142F8D110BD2C0000004C00000080
S31508007AC005020602060307030803090309040A0454
S31508007AD00B040C040C050D050E050F050F06100604
S31508007AE010071008FBECFFFFFC0000000C0000204C
S31508007AF0000000004BEEFFFF0C000000980000009D
S31508007B00000000200000000000F00DF8002801D059
S31508007B10FFF7C2FFAFF300800020AFF30080FFF746
S31508007B2039FD00F002F80120704700F001B80000A6
S31508007B300746384600F002F8FBE7000080B5AFF3C9
S31508007B400080024A11001820ABBEFBE7260002009F
S31508007B50024885460248804702480047080900202F
S31508007B60417A0008897B000802030405060708090C
S31508007B700A0B0C0D0E0F101000000000000000008C
S31508007B800102030406070809AFF30080AFF300807B
S31508007B90FFF7BAFF1000000000A24A040100000027
S31508007BA00000000001020304FFF7FEBFFFF7FEBF57
S31508007BB0FFF7FEBFFFF7FEBFFFF7FEBFFFF7FEBFEB
S31508007BC0FFF7FEBFFFF7FEBFFFF7FEBFFFF7FEBFDB
S31508007BD0FFF7FEBFFFF7FEBFFFF7FEBFFFF7FEBFCB
S31508007BE0FFF7FEBFFFF7FEBFFFF7FEBFFFF7FEBFBB
S31508007BF0FFF7FEBFFFF7FEBFFFF7FEBFFFF7FEBFAB
S31508007C00FFF7FEBFFFF7FEBFFFF7FEBFFFF7FEBF9A
S31508007C10FFF7FEBFFFF7FEBFFFF7FEBFFFF7FEBF8A
S31508007C20FFF7FEBFFFF7FEBFFFF7FEBFFFF7FEBF7A
S31508007C30FFF7FEBFFFF7FEBFFFF7FEBFFFF7FEBF6A
S31508007C40FFF7FEBFFFF7FEBFFFF7FEBFFFF7FEBF5A
S31508007C50FFF7FEBFFFF7FEBFFFF7FEBFFFF7FEBF4A
S31508007C60FFF7FEBFFFF7FEBFFFF7FEBFFFF7FEBF3A
S30908007C70FFF7FEBF4F
S70508007B89EE
